:020000040800F2
:10500000B81A0020D5500008E9860008ED7D000898
:105010000000000000000000000000000000000090
:10502000000000000000000000000000E190000807
:105030000000000000000000E98E0008DD9100087B
:10504000E7500008E7500008E7500008E750000864
:10505000E7500008515B0008E7500008E7500008DF
:1050600000000000E75000088D5A0008E7500008D3
:10507000E7500008D982000800000000E75000084F
:1050800000000000E75000080000000000000000E1
:10509000E750000800000000E7500008E750000853
:1050A000E7500008E7500008E7500008C59A0008DC
:1050B000E7500008E7500008000000000000000072
:1050C0000348854600F060FC00480047C9A8000876
:1050D000B81A00200448804704480047FEE7FEE76E
:1050E000FEE7FEE7FEE7FEE779920008C150000800
:1050F00030B50B46014600202022012409E00D4670
:10510000D5409D4205D31D469540491B25469540F7
:1051100040191546521E002DF1DC30BDF0B51FB40C
:105120000646002082B005464024019100901BE015
:10513000019922460F46304600F04EFB049A059B2B
:10514000801A994110D310461946224600F034FBCC
:10515000361A8F410197224601200021009F00F05E
:105160002BFB38184D4100902046641E0028DFDCE0
:10517000019B00982946324607B0F0BD03460B4319
:105180009B0703D009E008C9121F08C0042AFAD2FD
:1051900003E00B780370401C491C521EF9D2704783
:1051A000D2B201E00270401C491EFBD270470022BF
:1051B000F6E710B513460A4604461946FFF7F0FF16
:1051C000204610BD30B504460020034600E05B1CBD
:1051D000934203D2E05CCD5C401BF8D030BDF8B503
:1051E00002464A40D40F42004B0052085B089A42E4
:1051F00002D20246084611464A0023D0C30D4A0097
:10520000DDB2120EAD1A202D35DA49020126490A07
:10521000F6058A19002C00D0524220214F1B11465E
:10522000B9402A411018C20D9A4221D0002C17D043
:10523000012D08DCDA05801AD20F8019D207DBB203
:1052400000F0F6FAF8BDDA05801A012340001B06CB
:10525000C01880185A428018CA0F1043490007E04E
:105260004908C2071143DA05801A801940088018DE
:1052700000F0D6FAF8BD61000122511A001BF7E7D1
:105280000122D2075140AAE70122D2075040A6E7E7
:1052900070B502464A40D50F40004A00ED0740086D
:1052A0005208002814D0002A12D0C40DD30D410298
:1052B0000120C0055202490A520AE41A09181218BC
:1052C0007D34914201D3641C00E04900002C01DAD6
:1052D000002070BD0023914201D3891A0343400886
:1052E00049000028F7D100290AD0914202D10121BA
:1052F000C90705E0914201D2012101E00121C94322
:10530000E005C018401900F08BFA70BDF0B50746F3
:105310000846584087B0C00F049048000E46590018
:1053200040084908BC1A884105D2384631461E4615
:1053300017460B4602465800400810434CD0300D2B
:10534000039040055900400D490D0590401A029008
:10535000402872DA18030121000B09050843019067
:1053600004980092002805D00199524200208841FB
:1053700000920190029840210A1A0199009800F0C9
:105380001BFA05460C466B4607CB00F036FAC019EF
:105390007141039A0E0D0023D71756401A467A40E2
:1053A000164344D0049A002A2DD0029A012A039A67
:1053B00015DC1205C01A914101263605001C714109
:1053C000D20F059ED2070093019202962A462346E9
:1053D00000F074FA07B0F0BD38463146FAE716051A
:1053E000224A0F46B218C01AB74101210905001C14
:1053F0004F4100187F41114618187941E20F1043C0
:105400006D19644113E0E2076D0815436408C20793
:105410001443039A01261205C01A91413605001C57
:105420007141CE07400830434908C01851412A460F
:10543000234600F036FACDE7FFE70498012240004A
:10544000C117121A00238B4104983146C417381A29
:10545000A141EEE730B40124E407634030BC55E7D6
:1054600030B40124E407614030BC4FE70000E0FFA6
:10547000F0B51FB488B00B990998002448400999E9
:10548000C00F490049080991C0070B9900904900D5
:1054900049080B9109990898A64608431CD00B9916
:1054A0000A98084318D0099801244000420D48008A
:1054B000410D099824050003000B204309900B9827
:1054C0000003000B20430B9050181C494018002289
:1054D00001901446104605E0002001460DB0F0BDD5
:1054E000032801DA034600E003239C46C11A0AAEF2
:1054F0000AE05F0008ADED5B4F00F75B7D430027DE
:10550000AA187C41491C5B1E6145F2DD410004ABD9
:105510005A522104120C0A43240C401C0828DFDBD9
:10552000019802900099704601910090059B049AA1
:105530000799069800F0C2F9D0E700000DFCFFFFC4
:10554000F0B50C465C4085B0E40FE40703944C00D2
:1055500000266408590094464908024602962243F0
:1055600021D062460A431ED06200570D4A000E0346
:105570002303550D012402462C492405781B1B0BDF
:10558000360B401823432643614600901C46501AB0
:10559000B44103D30098401C009002E09218009898
:1055A0005B41002803DA0020014605B0F0BD002071
:1055B000012109050746864611E064461D46141B75
:1055C000B54106D36546521BB341744607430C43AD
:1055D000A646CD0740084908284392185B41054676
:1055E0000D43EAD11046184313D060461946504087
:1055F0007140084306D06046101AB34106D201221A
:10560000002306E000220123DB0702E00122D2434F
:105610005310009874460105381C6141029C039D9B
:105620000019694100F03DF9BFE70000FD030000EB
:10563000C217C10F504010B54018CA079623002169
:1056400000F0F6F810BD10B500229623114600F0C8
:10565000EFF810BD0EB5C217C10F5040CA07401871
:105660000021054B0293019200910A460B4600F07F
:1056700025F903B000BD0000330400000EB5054954
:105680000291002100910A460B46019100F016F9A3
:1056900003B000BD33040000410040020122400A73
:1056A000D205090E80187F2901DA0020704796295B
:1056B00003DC9622511AC8407047963988407047DB
:1056C00070B5CD0F4A0009030123090B1B051943CF
:1056D0000B4BED070024520D9A4201DA002070BDF9
:1056E000074B34339A4203DC9A1A00F075F802E053
:1056F0000449511888402C43F1D0404270BD00004D
:10570000FF030000CDFBFFFF4A0009030123090B43
:105710001B051943094B10B5520D9A4201DA0020BE
:1057200010BD064B34339A4203DC9A1A00F054F849
:1057300010BD03495118884010BD0000FF03000050
:10574000CDFBFFFFC20FD207400040080BD0C10DB8
:105750000723DB01C91840020905400A1143C208AA
:10576000400711437047002001467047CB0FDB070D
:10577000490010B5490802460A4307D00A0D07241C
:105780000903E401090B121B002A01DC002010BDF3
:10579000C900440F0C43C100E018D205801800F086
:1057A0003FF810BD0122D207002800DB101A0029A3
:1057B00000DB511A8142704710B5202A04DB0146F4
:1057C000203A9140002010BD914020239C1A0346AE
:1057D000E3401943904010BD10B5202A04DB084671
:1057E000203AD040002110BD0B46D340D0402024A9
:1057F000A21A91400843194610BD10B5202A06DBB5
:10580000CB170846203A1041C1170B4306E00B4660
:105810001341D0402024A21A91400843194610BDDC
:10582000002904DA401C490001D1400840007047BB
:1058300070B40024050C05D11024000402D1002905
:1058400021D01124050E01D100020834050F01D129
:105850000001241D850F01D18000A41C002801DB5C
:105860004000641C002908D020252E1B0D46F54061
:10587000A14000D001212943084301061B1B000A57
:10588000DB1D02D5002070BC7047DB05181880189E
:105890000029F8DA401C4900F5D170BC40084000EE
:1058A000704710B5002B08DA0024401C61419218A3
:1058B0005B411A4301D14008400010BDF0B51FB450
:1058C00082B005460C0003D0084604F0D3F902E08C
:1058D00004F0D0F920300246009021462846FFF718
:1058E0006BFF049B059A04460F4618431143084377
:1058F00014D0184610431BD0009840210A1A1846AD
:105900000599FFF769FF05460E46009A0599049828
:10591000FFF752FF084305D0012004E02046394636
:1059200007B0F0BD0020C11705430E432C43374399
:1059300000990E986305401A7905E40A00220C4389
:10594000FD0A0A3002D500200146E9E701051019D9
:1059500069410C9C0D9D00196941FFF7A2FFDFE72B
:1059600010B5002904DB0124E40740428C412146A4
:10597000002B04DB1C460123DB075242A341994262
:1059800000D1904210BD0000064C0125064E05E0F6
:10599000E36807CC2B430C3C98471034B442F7D350
:1059A000FFF792FB40AE000860AE000838B5044631
:1059B000064805490068FFF79BFB604300E0401E76
:1059C00000900028FBD138BD40420F001401002098
:1059D000F8B50446006881688907890F012902D15A
:1059E0000168C90722D18168114A1026114001259A
:1059F00000290ED18168294381600120FFF7D6FF7D
:105A000000F0C8FF07460CE000F0C4FFC01B0A28E6
:105A100007D9606D30436065A06D2843A065012003
:105A2000F8BD20680068C043C007EDD10020F8BD74
:105A30001700008010B5012005F01CF80A4C13284F
:105A4000A0700AD0E01C02F0FBFBE078A0703328C5
:105A500006D006490020C88710BD05F043F810BDE8
:105A600002F0C0FB10BD000000000020480D002027
:105A700010B500231A4603E0845CE3189BB2521C65
:105A80008A42F9D3D84380B210BD000010B5034854
:105A900000F036FD024800F033FD10BD581600201E
:105AA0001016002030B5446C1C252C400125A54063
:105AB000046C6560046863608368102B036803D01E
:105AC00099600068C26030BD9A600068C16030BDF6
:105AD00010490120487202205E31487203203C398F
:105AE000487204200E3948720A4B0B495A1C087838
:105AF0005871497899712333187159712033187787
:105B00005977107551751A461E32107551751076F9
:105B10005176704748110020FC00002010B503F0BA
:105B2000B5FA202003F050FB012004F053FC0020C4
:105B300003F04AFB044804F0F1FA044804F09AFD2B
:105B4000002004F0CFFD10BDC000002083800000C5
:105B500070B505200121000700F010FF00240D4D55
:105B6000002800D02C6002210B4800F007FF00281D
:105B700008D10A482C6000880A2148430849088057
:105B800003F0CCFF012000F031FE022000F02EFED9
:105B900070BD00000C01002000040050E600002051
:105BA000F80000207047000010B5084900224A6143
:105BB00007494B684C1523434B604B68082423432B
:105BC0004B60C009C001026010BD0000A01600209B
:105BD000002002407FB500250C460646039500F0E4
:105BE000D5FDE009029003A901960095684600F0F2
:105BF00065FD002804D000F09DFD002004B070BDBC
:105C000000F098FD0120F9E710B5002302E0C45C24
:105C1000CC545B1C9342FAD310BD000010B5214A4E
:105C200000219069C305204804D541690223194326
:105C30004161911593699B0505D54369012423436F
:105C400043616302194393695B0505D543690824E1
:105C500023434361E301194393691B0505D5436958
:105C60000424234343616302194393699B0405D5CC
:105C700043691024234343616302194393699B03DF
:105C800004D5446920231C43446119439369DB0311
:105C900005D54369402423434361A0020143916138
:105CA00010BD000000200240A016002070B505467F
:105CB00000F070FE0646184C0AE0681C08D0002D63
:105CC00004D000F067FE801BA84201D9032070BDFC
:105CD000A069C007F1D1A069800701D50220A061A9
:105CE000A069C00511D4A06980050ED4A069400543
:105CF0000BD4A069000508D4A069800405D4A0696C
:105D0000800302D4A069C00303D5FFF787FF0120F9
:105D100070BD002070BD000000200240F8B517469D
:105D2000002605460C4600F031FD09E02946022018
:105D3000226800F00DFD002804D1241D2D1D361D04
:105D4000BE42F3D300F0F6FCBE4201D20020F8BD03
:105D50000120F8BD10B5084902460020054B4979DD
:105D600005E044001C5B944203D0401CC0B2884252
:105D7000F7D310BD8A1200206000002010B509483A
:105D800000F0C6FF80B2FFF779FC074A074BFFF728
:105D90006FFB0022064BFFF7D3FBFFF7B5FC80B289
:105DA00010BD0000CC140020F853E3A59B843E40B6
:105DB00000408F40F8B5414CE079002801D0002028
:105DC00000E00120E0713D493D48CA790275097A39
:105DD00041753C490A780276497841763A4801781B
:105DE00037481330017005214172962004F032FCCF
:105DF0004B20C00004F048FC3149002213310C2034
:105E000004F012FD00210C2004F020FD022004F01B
:105E100071FC2E4D00210F2004F096FB2842E06219
:105E2000F8D0E06A411C3BD0294E2A4F400439D5B6
:105E30008122D20100210F2004F0CBFC0021102090
:105E400004F082FB41061E48490E0022633004F034
:105E5000B1FB1B4D6335687A052820D10222194910
:105E6000681DFFF7AFF9002819D1A87A60711348AF
:105E70000422691C4030FFF781F9206C00F02EF8F5
:105E8000A0836079294642000B3108467330FFF742
:105E900075F9A08B31884843388002202070F8BD06
:105EA00002F046FC0C480188A08B0546FFF720F95C
:105EB0003088414339806D1EA583F8BD6000002005
:105EC000A9110020FC000020D600002000D02724CB
:105ED000E0000020DE000020E200002010B50446B3
:105EE0000E4800F015FF0E49C006C00E098805E0F7
:105EF0002246C240D2070FD0401CC0B28842F7D31E
:105F0000012005E02246C240D20705D0401CC0B2A5
:105F10008842F7D3491EC8B210BD0000CC1400203F
:105F2000E200002010B5084800F096FA0A21064861
:105F300000F032FA044800F01DF9800503D502484C
:105F400000F01AF980B210BD70140020F8B52F4D82
:105F500000220121284600F016FDFFF7E3FFFFF7BE
:105F600072FB2B4E3146FFF793F92A4C0122A060B9
:105F70001146284600F007FD2749A0680025884201
:105F80003EDB2078254F002815D02570FFF7CAFF8B
:105F9000FFF759FB3146FFF77BF9A060FFF7D2FB13
:105FA00000223B46FFF756FA00221D4BFFF760FA2E
:105FB000FFF7DCFB6060A068FFF7C4FB00223B46F4
:105FC000FFF748FA174A184BFFF752FA06460F46F2
:105FD0006068FFF7B7FB134A144B5242FFF748FAC9
:105FE00032463B46FFF792F9FFF7C0FB104960606D
:105FF000884201DD616004E0FF21C905C84200D389
:1060000065606068FFF748FBC0B2F8BD000400504F
:1060100000401B443C0000200000604000000C4099
:1060200000E064403333333333B33040CCCCEC3F07
:106030000000C842F8B5054604464035287C0026D5
:10604000012808D001202874206881688907890FF9
:1060500001290ED101E00220F8BD0168C90708D06E
:10606000606D2021084360650126002028743046B9
:10607000F8BD616DFF220132914302221143616537
:10608000C1688907890F0091C16889088900C160CA
:106090002068816892071143816000F07BFC07460D
:1060A0000EE000F077FCC01B0A2809D9606D0221C0
:1060B0008843102108436065002028740120F8BD42
:1060C000206880680028ECDB2068C168009A1143D2
:1060D000C160606D80088000401C6065C5E70000FD
:1060E000F8B506460D464036317C01290DD0012118
:1060F000317401688A68520709D5416D2022114325
:106100004165002030740120F8BD0220F8BD174B16
:106110006A68D80547109A42154C8A6A2B6812D0D3
:106120005B035B0B1A438A622968490305D5A168A2
:106130000143A1600A20FFF739FC2868800312D5CB
:10614000A06838430EE05B035B0B9A438A622968C0
:10615000490302D5A1688143A1602868800302D564
:10616000A068B843A06000203074F8BD01100000A2
:1061700000270140406D70470068006C70470000C8
:1061800070B5040006D0606D264600254036002814
:1061900002D006E0012070BDA5653574204600F0F0
:1061A000D3F8606DC00603D421688868400705D520
:1061B000606D1021084360653574EBE7606DFF2268
:1061C0000132904302221043606588688207920F73
:1061D0005B48012A02D10A68D2072BD103236268E7
:1061E0009B079A4205D05B429A4202D05B009A42DA
:1061F00009D10A69920092080A6121680A696368F4
:106200001A430A610CE00A69920092080A618168E7
:106210000F2292049143816081686268114381601A
:106220002168CA6818239A43CA602168CA68A368AB
:106230001A43CA60816801225206914381608168D5
:10624000A28E52061143816020688168C90004D47F
:10625000816801221207114381602068C168394AB0
:106260001140C1602069E168022825D00020014367
:10627000204620300278037B52035B001A4311430F
:10628000226B1143A26992031143E269D2031143C5
:106290002268D3681943D160616A0A46FF3AC23A5C
:1062A00005D0A26A11432268D3681943D1604278AD
:1062B0000121012A02D00BE00420D8E70078002851
:1062C00023D0606D202210436065A06D0843A06557
:1062D000E06B012820681FD00169C90703D001695C
:1062E00049084900016120684169C908C900416144
:1062F00020684169A26B11434161A565606D80080A
:106300008000401C6065002070BD2068C2680123C9
:106310001B041A43C260DBE70269FF239B009A4318
:10632000026120680269236CA66C1A43636C3343D4
:106330001A430261206802690A430261D3E7000040
:10634000002701401902FEFF10B586B00446142153
:106350006846FEF72CFF0E492068884216D10D488A
:10636000416B421511434163C16A01221143C1626D
:10637000C06A6946104005900220009003200190F9
:10638000002002900520000700F03CFA06B010BD86
:106390000024014000100240F8B50446406925463B
:1063A00040350E4608280BD02068C068C00709D0C9
:1063B000606D202108436065002028740120F8BD2D
:1063C000082700E00C2700F0E5FA009011E0701CAF
:1063D0000FD0002E05D000F0DDFA0099401AB0422F
:1063E00007D9606D042108436065002028740320EC
:1063F000F8BD206800683842E9D0606D012149028B
:10640000084360652068C16809058A0F0C21002ACD
:106410001BD12022125D002A17D10268120714D561
:10642000826853070122002B08DB43688B434360DB
:10643000606D130298431043606506E0606D202391
:1064400018436065A06D1043A065A069002801D1C4
:10645000206801600020F8BD70B504462168002066
:106460008968490721D425464035297C01291CD05B
:1064700001212974E169012904D02046FFF7A8FA17
:10648000002811D1616D0A4A1140FF2201321143E7
:1064900061650021A165297422681C2111602168B1
:1064A0008A6804231A438A6070BD022070BD000010
:1064B000FEF1FFFF70B50024014620314A79022A1F
:1064C00003D00421C163012418E0026813680E257B
:1064D000AB431360026813685B085B001360436C96
:1064E0001C221340012215469D40036C5D604A71D9
:1064F00000220A71816B002900D08847204670BDB8
:10650000F0B4016C0D6801680C68466C1C23042211
:106510001E401746B7402F420ED067070CD50C68B7
:10652000A40602D40C6894430C60416C19408A4064
:10653000016C4A60016B1AE00227B74002462F4007
:106540002032002F17D0A70715D50C68A40605D454
:106550000C680A25AC430C6001215171446C022186
:106560001C40036CA140596000211171C16A0029CF
:1065700018D0F0BC08470827B7402F4212D0240794
:1065800010D50C680E25AC430C60446C01211C40F6
:106590000B46A340046C6360C1635171002111710B
:1065A000416BE4E7F0BC704770B504003CD01F4875
:1065B000256814212818FEF79BFD800060641C48A4
:1065C0002064022120462030024641712968194882
:1065D000E3680140A06866691843236933431843A0
:1065E000A3691843E3691843236A184308432860E2
:1065F0000121A0688903884210D00D488030836A49
:10660000656C1C210D400F26AE40B3438362656C60
:1066100063680D40816AAB400B4383620020E063F6
:1066200001215171107170BD012070BDF8FFFDBFD7
:10663000000002400F80FFFFF8B504468C46203072
:1066400001790025012909D0012606714179002729
:10665000012905D0077102252846F8BD0220F8BDA2
:1066600002214171E763206801684908490001601F
:1066700061462046FFF716FA206B00282068016863
:1066800001D00E2205E004229143016020680168D8
:106690000A22114301602068016831430160DBE791
:1066A00070B5044600F076F90546601C00D0641C05
:1066B00000F070F9401BA042FAD370BDF8B51A4E35
:1066C0000546307C0F46012807D00120307417485A
:1066D000FFF7ECFA010002D021E00220F8BD002013
:1066E000C04338606C6814E02046FFF75DFA0F483D
:1066F000FFF7DCFA01460E48426808239A434260DD
:10670000426843159A434260002901D03C6006E08C
:106710008034A8686A68C0018018A042E4D80020CC
:1067200030740846F8BD0000A016002050C30000D9
:10673000002002400548416802221143416041683F
:1067400001221143416000207047000000200240F8
:10675000F8B50C4C1646207C0F46012808D00120C5
:1067600020740948FFF7A2FA0025002802D006E0AD
:106770000220F8BD65613E600348FFF797FA257473
:10678000F8BD0000A016002050C300001148416869
:10679000C9070BD0EFF3108172B60F4AC2600F4ADF
:1067A000C26081F310884168C9070ED1416889072A
:1067B0000DD5EFF3108172B6094A0261094A0261F0
:1067C00081F310884068800701D5012070470020C0
:1067D0007047000000200240EFCDAB8905040302A2
:1067E000BFAE9D8C161514137047000010B50449F8
:1067F0004A69024202D04861FFF7F6FF10BD00006F
:1068000000040140F8B500230124A2E027469F4080
:106810003A4070D04D68022D01D0122D14D1DD0800
:10682000AD002D1800952D6A5E07AC46F50E0F26BB
:10683000AE46AE406546B543AC460E697546AE40C1
:1068400065462E43009D2E624D68012D05D0022D18
:1068500003D0112D01D0122D16D185680326AC4628
:106860005D00AE46AE406546B543AC46CE68754663
:10687000AE4065462E43866046680D79BE43ED0600
:10688000ED0F9D403543456006685F000325BD4020
:10689000AE46AE430D79B446AE07B60FBE40654670
:1068A0002E430660C6687546AE438D68BD403543CD
:1068B000C5604D68ED004BD5294D6E6B26436E6368
:1068C0009E08284DB6007519AC46AD689E07360F78
:1068D0000F27B740BD4305273F07B84201D1002726
:1068E00015E0214FB84201D1012710E01F4FB842F7
:1068F00002D102270BE02BE01D4FB84201D1032744
:1069000005E01C4FB84201D1052700E00627B7403B
:106910002F436546AF60184D2E684F689643FF03BE
:1069200000D516432E606E684F689643BF0300D5AE
:1069300016436E60AE684F689643FF0200D516435B
:10694000AE60EE684F689643BF0200D51643EE6016
:106950005B1C0A681546DD4000D057E7F8BD000013
:1069600000100240000001400004005000080050E8
:10697000000C0050001C0050000401400069084059
:1069800000D001207047002A01D0816170478162E8
:1069900070470000014800687047000010010020A7
:1069A00002480168491C0160704700001001002086
:1069B00010B50848002401684022114301602046B8
:1069C00000F00AF8002801D0012401E000F0CCF921
:1069D000204610BD0020024070B5054609487D21C3
:1069E0000024C9000068FEF783FB00F061FE002868
:1069F00001D0012404E000222946501E00F0D4F901
:106A0000204670BD1401002070477047F8B53A4C1D
:106A100001266078401C6070E670208C401C208449
:106A2000608902F09BFB354FF888FEF70CFE344975
:106A3000FEF72EFC334D00902968FEF7D0FB28604E
:106A4000E16AF005814203DB0098FEF71DFCE0627D
:106A500002212D48FFF792FF002808D00020206374
:106A60002A492F682A488F4227DD067027E0F888D8
:106A7000FEF7E9FD2249FEF70BFC216BFEF7AFFBA9
:106A8000244920638842EBDBE079002813D0002101
:106A90001A484030818004F03DF90121002289022A
:106AA0001948FFF770FF7D200001FFF7F9FD1B4932
:106AB0001948C860D4E70121EAE700210170207A73
:106AC000401EFEF7B5FD3946FEF76CFE06D820796C
:106AD000002803D01248C1793143C171207AFEF7F2
:106AE000B2FD2968FEF75EFE04D22079002801D0AD
:106AF00003F084FFF8BD0000D4000020480D002002
:106B000000007A440C0100200004005000004040C6
:106B1000660000200000A0400400FA0500ED00E03F
:106B2000BC110020704770B505000DD002202C4626
:106B30002034A073284601F0D7FB284600F0BEF8A9
:106B40000020A073607370BD012070BD7047704756
:106B500010B5044600680168C943C90708D18168B7
:106B6000C943C90704D1012141602046FFF74EFF08
:106B700020680168C943890708D48168C943890727
:106B800004D4022141602046FFF73EFF20680168DF
:106B9000C943490708D48168C943490704D404217B
:106BA0004160204600F0DEF820680168C94309070B
:106BB00008D48168C943090704D4082141602046EC
:106BC000FFF7B0FF20680168C943C90608D481688F
:106BD000C943C90604D4102141602046FFF715FFC0
:106BE00020680168C943890608D48168C9438906B9
:106BF00004D4202141602046FFF7A9FF20680168E6
:106C0000C943490608D48168C943490604D44021D0
:106C100041602046FFF79AFF10BD0000F8B5040060
:106C200005D025462035A87B002802D006E00120AB
:106C3000F8BD00206873204600F052F80220A873C7
:106C40002068C26884466368012B04D00120A16AD1
:106C5000C005814201D11E208243154861698142ED
:106C600001D0144802401448A66802401846304338
:106C7000676A266A3E433043A66A30431043012BBD
:106C800003D00122D205964203D12369E2681A4358
:106C90001043074A914205D0A2691143E2690243B9
:106CA000084610436146C8600120A8730020F8BD63
:106CB000FFFF00003F1FFFFFF8F119FF10B500684C
:106CC0000549884207D10548816B4900490881631D
:106CD0000D2000F055F810BD007C0040001002406F
:106CE00010B50068084988420CD10848816BC2047D
:106CF00011438163002201210D2000F055F80D2081
:106D000000F048F810BD0000007C00400010024078
:106D10000068C0697047000070B502240346203344
:106D20009C730F4C2568E604354325600468E568CC
:106D3000B6123543E5600568AE6801242643AE60AF
:106D400005682E6926432E610568A96101684A61BC
:106D5000006801690422114301619C73002070BD29
:106D600000040140704700000448416B01221143B8
:106D70004163816B0204114381637047001002403C
:106D8000C106C90E01208840014908607047000013
:106D900080E100E0C106C90E012088400149086079
:106DA0007047000000E100E010B501F09FFC10BD4D
:106DB00002494A6882434A60704700000070004000
:106DC000024801688215114301607047007000405D
:106DD00002494A6802434A60704700000070004060
:106DE0000548016802221143016004480169042238
:106DF0001143016130BF70470070004000ED00E0BA
:106E00000A4B1A689208920002431A600848036904
:106E1000042213430361012906D040BF20BF20BFD5
:106E2000016991430161704730BFF9E7007000408C
:106E300000ED00E0F8B504460078544D800672D5A8
:106E4000524E0027403EB06BC00004D4B06BA90581
:106E50000843B06301274E480168C90511D4016891
:106E6000821511430160FFF795FD009005E0FFF7E3
:106E700091FD0099401A642837D845480068C0053C
:106E8000F5D532680321090560680A400140914246
:106E900008D08103890F032904D13168890301D502
:106EA0000120F8BD2A69032109040A4022D00840C4
:106EB00090421FD0207880061CD528692A69884313
:106EC0000121C9040A432A612A698A432A61286187
:106ED000C0050FD5FFF75EFD009008E0FFF75AFDF3
:106EE0000099411A2B48814201D90320F8BD286935
:106EF0008005F3D561688803800F032805D13268C7
:106F00000005824301400A43326028690322616818
:106F10001204114008432861002F04D0B16B0120F6
:106F200000078143B1632078C00705D0E868A168F5
:106F3000800880000843E8602078800705D5E8686D
:106F40000C218843E1680843E8602078400706D5B3
:106F5000E86803218902884321690843E8602078B2
:106F6000000706D5E86803210903884361690843DF
:106F7000E8602078000606D5E86803218904884384
:106F8000A1690843E8600020F8BD000040100240FD
:106F90000070004088130000F8B50E4605007DD053
:106FA00053480068C007C00FB0420AD25048016879
:106FB00049084900314301600068C007C00FB04272
:106FC00071D128784B4C800705D5E068F0218843C3
:106FD000A9680843E0602878C00752D06868022892
:106FE00017D0032818D02168012818D08905002956
:106FF00059DAE168890889000143E160FFF7CAFCBA
:1070000069680746022912D003291CD0012926D01D
:1070100033E021688903EAE721688901E7E7490746
:10702000E5E7FFF7B7FCC11B3348814223D8E0688E
:107030000007800F0228F4D123E0FFF7ABFCC11B4F
:107040002D48814217D8E0680007800F0328F4D14B
:1070500017E0FFF79FFCC11B274881420BD8E0686F
:107060000007800F0128F4D10BE0FFF793FCC11B50
:107070002148814201D90320F8BDE0680007800F54
:10708000F3D11B480168C907C90FB1420DD9016886
:107090004908490031430160006800E003E0C0078F
:1070A000C00FB04201D00120F8BD2878400706D5B6
:1070B000E068072109028843E9680843E06028780E
:1070C000000707D5E0680721C90288432969C9007C
:1070D0000843E06000F036F8E168084A0906090F45
:1070E000515CC840064908600020FFF775FCF8BDF8
:1070F0000020024000100240881300001EAE00086D
:1071000014010020044805490068C968044A49057B
:10711000490F515CC8407047140100200010024024
:1071200037AE0008044805490068C968044A890464
:10713000490F515CC8407047140100200010024004
:1071400037AE000810B5184AD1680C200840042852
:107150000BD0082810D00C2810D050680004410F24
:107160000120C003491C884010BD1068C00601D52D
:107170000E4810BD0E4810BD0E4810BD88020E4BC3
:10718000000F185C0902D368890F491CDB0301D585
:10719000084A05E01268D20601D5044A00E0044A14
:1071A0005043FDF7A5FF10BD0010024000093D004F
:1071B0000024F40000127A002EAE0008FEB505008F
:1071C0007ED0FE4CE7680C20E668074001200004F2
:1071D00006402878C00747D0082F05D00C2F0AD1C9
:1071E00001200004864206D1206880033CD56868EF
:1071F0000028E5D038E0012069680004814203D10D
:1072000021680143216011E0052301221B0492043F
:107210009942216802D111432160F1E78143216045
:107220002168014000912068904320606868002830
:107230000DD0FFF7AFFB009005E0FFF7ABFB009927
:10724000401A64287AD820688003F6D50CE0FFF74E
:10725000A1FB009005E0FFF79DFB0099401A642810
:10726000F0D820688003F6D42878800755D5092304
:10727000E868042F0DD00C2F01D1002E09D0002872
:107280003BD02168994301432160FFF783FB064609
:1072900027E02168490701D5002891D061681F22A5
:1072A000120291432A6912021143616021689943D5
:1072B00001432160FFF746FFE16809060A0F00E07D
:1072C00079E1BF49895CC840BE4908600020FFF7EA
:1072D00083FB002872D120E0FFF75CFB801B0228B3
:1072E000B0D820684007F7D560681F21090288439D
:1072F00029690902084360600FE0206840084000E7
:107300002060FFF747FB064604E0FFF743FB801BC6
:10731000022897D820684007F7D42878C0065FD5A0
:10732000002F0CD0A869002849D02068FF21013126
:1073300008432060FFF72EFB06462DE0C0E02068E2
:10734000800502D5A8690028A7D0606807214903F5
:107350008843296A084360606068297F0002000A48
:10736000090608436060286A410B0120C003491CDC
:107370008840E16809060A0F9149895CC840914933
:1073800008600020FFF728FB002817D128E0FFF74E
:1073900001FB801B0228A3D820688005F7D5606810
:1073A000072149038843296A084360606068297F90
:1073B0000002000A09060843606011E0E1E021686C
:1073C000FF20013081432160FFF7E4FA064604E024
:1073D000FFF7E0FA801B022872D820688005F7D4F6
:1073E0002878794E000724D568690028306910D0C4
:1073F000012108433061FFF7CDFA009005E0FFF767
:10740000C9FA0099401A02285AD830698007F6D57F
:107410000FE0400840003061FFF7BCFA009005E043
:10742000FFF7B8FA0099401A022849D83069800756
:10743000F6D42878400765D500200290A06BC000E4
:1074400006D4A06B012109070843A0630120029024
:107450005E480168C90511D40168821511430160B5
:10746000FFF798FA009005E0FFF794FA0099401AA8
:10747000642825D855480068C005F5D5FF20AA68BE
:107480000130824203D131690143316111E00121B0
:107490008902002A07D005231B029A4203D13269D0
:1074A0000A433261EFE732698243326130698843CF
:1074B0003061A86800280FD0FFF76CFA009007E051
:1074C0005EE0FFF767FA0099411A4148814257D8B8
:1074D00030698005F5D50DE0FFF75CFA009006E015
:1074E000FFF758FA0099411A3948814248D8306963
:1074F0008005F5D40298002804D0A06B012109076B
:107500008843A063686A002864D00C2F3ED001260F
:1075100036060228206805D0B0432060FFF73AFA0B
:1075200005462FE0B0432060FFF734FA074604E039
:10753000FFF730FAC01B022822D820688001F7D458
:10754000E96AA86AE2680843296BFD231B049A4391
:1075500011430843E060206830432060FFF71AFAC7
:10756000054604E0FFF716FA401B022808D82068F9
:107570008001F7D52EE0FFF70DFA401B022801D954
:107580000320FEBD20688001F5D423E00128F8D057
:10759000E06801210904AA6A014091420BD10F2140
:1075A0008904EA6A0140914205D103218905084016
:1075B000296B88420ED00120FEBD00000010024061
:1075C0001EAE000814010020401002400070004070
:1075D000881300000020EFE770B5040007D00026F4
:1075E00025464035A662687C002802D005E00120CF
:1075F00070BD2E74204600F02FF8022068742068B9
:107600000168402291430160A168606822690843D3
:10761000E16811430843616901220843A1695202EC
:1076200011400843E1690843216A0843A16A0843FD
:1076300021680860A0690421000C0840616A0843C1
:10764000216848602068C16992009143C161666504
:1076500001206874002070BD10B586B00446142166
:107660006846FDF7A4FD10492068884219D10F48EB
:10767000416B821411434163C16A01221143C1620B
:10768000C06A002110400590E02000900220019087
:107690000320039002910491052069460007FFF73B
:1076A000B1F806B010BD00000030014000100240EB
:1076B000094910B5401E884201D9012010BD074C70
:1076C00060610321081F01F011F80020A06107206C
:1076D0002061002010BD0000FFFFFF0000E000E07F
:1076E000F0B502462032137E012B15D00127177604
:1076F0000223537605686C68AB687026B4430E6845
:10770000496826438024A34319436E600068816062
:10771000577600201076F0BD0220F0BD70B5040051
:1077200005D025462035687E002802D006E00120DD
:1077300070BD00202876204600F00AF80220687606
:10774000211D206801F0C4FD01206876002070BD75
:10775000006801218907884204D10348816B012216
:10776000114381637047000000100240F8B50546E0
:1077700004462035287E012817D001262E760220C7
:107780006876226890687727FF23B8431B029843E6
:1077900090600A68502A31D00EDC202A4BD006DCDB
:1077A000002A48D0102A3AD145E00220F8BD302AFC
:1077B00041D0402A33D136E0602A27D0702A12D037
:1077C00001200003121A2AD0824228D1CB684A68CD
:1077D0008968206801F0B5FD206881680122920364
:1077E000114381601BE0CB684A688968206801F01A
:1077F000A8FD216888683843886010E0CA68496835
:10780000206801F018FE5021206806E0CA68496827
:10781000206801F021FE6021206801F09DFD6E7658
:1078200000202876F8BDCA684968206801F003FE88
:1078300040212068F1E711462068EEE710B586B0D8
:10784000044614216846FDF7B2FC0121206889072F
:10785000884212D10A49CA6A02200243CA62C96A2E
:107860000190014005914102009100210291039194
:10787000049069460348FEF7C5FF06B010BD00003E
:107880000010024000040050F8B5064604462036B9
:10789000307E0D4601280DD0012030760220707612
:1078A0000427002A08D0042A16D0082A2AD00C2A35
:1078B0004DD137E00220F8BD206801F055FD206869
:1078C000816908221143816120688169B94381611E
:1078D00020688169EA6812E0206801F05DFD206897
:1078E00082690121C9020A438261206881690122FB
:1078F00092029143816120688169EA681202114312
:10790000816124E0206801F060FD2068C2690821DF
:107910000A43C2612068C169B943C1612068C16975
:10792000EA6812E0206801F06BFD2068C16901225D
:10793000D2021143C1612068C269012189028A43D0
:10794000C2612068C169EA6812021143C161012065
:10795000707600203076F8BD70B5040005D025465D
:107960002035687E002802D006E0012070BD00208E
:107970002876204600F00AF802206876211D20684B
:1079800001F0A6FC01206876002070BD704710B59C
:1079900004460068012201F0C7FC2068816849079D
:1079A000490F062903D0016801221143016000201C
:1079B00010BD000010B504460068002201F0B4FCC0
:1079C0002068016A054A114203D10168490849004B
:1079D0000160012020346076002010BD11110000EC
:1079E00070477047F8B502680446D069116893681B
:1079F00005072D0F5BD0DD07ED0FFF2621360E406A
:107A00002E4367D0C60706D0CE0504D501261662E0
:107A1000E26F3243E267870702220426002F06DA6C
:107A2000DF0704D027683A62E76F3743E767470705
:107A300006D5DB0704D023681E62E36F1343E367B8
:107A4000020709D520220A402A4305D023680822CC
:107A50001A62E36F1343E367E26F002A2FD08006B8
:107A600006D5880604D5216E002901D02046884716
:107A7000E06F21688968490601D4000724D52046B3
:107A800001F090FE20688168490619D5816840227E
:107A900091438160E06E002812D020498163E06E3E
:107AA000FEF708FD00280AD0E06E816B06E085062F
:107AB00010D58D060ED5216E1CE020468847F8BDF6
:107AC0002046FFF78EFFF8BD2046FFF78AFF002013
:107AD000E067F8BDC50208D55B0206D501200005A8
:107AE00010622046FFF77CFFF8BD030605D50B06A4
:107AF00003D5616E0029E0D1F8BD4006FCD54806EB
:107B0000FAD51368204640218B431360202161671A
:107B10000021616600F069F9F8BD000001970008D6
:107B200010B5040003D0606F002802D007E00120E8
:107B300010BD002170200155204600F027F82420B8
:107B4000606720680168490849000160204601F02B
:107B500073FE0128ECD0606A002802D0204601F0B4
:107B6000B1FC206841680922D2029143416020683B
:107B700081682A22914381602068016801221143B3
:107B80000160204601F004FD10BD0000F0B587B093
:107B9000064614216846FDF70AFB2C4930688842E6
:107BA00051D12B48416B0122920311434163C16AB9
:107BB00001221143C162C06A0025104005900320D4
:107BC000400200900220032701A9A1C104200490D3
:107BD000052069460007FEF715FE1F4C1D48A560ED
:107BE000E56081C48027E560A76020202561606191
:107BF0000002A0611848083CFEF7D6FC002801D01E
:107C0000FDF7D0FFF466A662144C124821461438E2
:107C100020600320606010200831A1C16561A5616A
:107C2000E56120462562FEF7BFFC002801D0FDF784
:107C3000B9FFB466002201211B20A662FFF7B4F849
:107C40001B20FFF7A7F807B0F0BD00000038014087
:107C5000001002403000024010160020581600208C
:107C6000F8B50446806F20284DD100290BD0002A9A
:107C700009D00123A0681B03984206D1206900287F
:107C800003D1C80701D00120F8BD25466035287C06
:107C9000012838D00120287458206165025300263D
:107CA000E6672220A067E06E002819D01749C1625C
:107CB000E16E17480863E16E16484863E06E1346AC
:107CC0008663676D21683A462431E06EFEF7B4FCA6
:107CD000002805D01020E0672E7420206067D2E7CE
:107CE0002E7420680168FF22013211430160206870
:107CF000816801221143816020688168402211431C
:107D000081600020F8BD0220F8BD00005D970008EA
:107D10009B9700081597000870477047FFB5044609
:107D2000406F83B017460D4620285CD1002D0AD045
:107D3000002F08D0A168C001814207D12069002826
:107D400004D1E80702D0012007B0F0BD2046603022
:107D50000290007C012846D0029801210174002085
:107D6000E06721206067FEF715FE26464036019049
:107D7000378277820120A1680003814202D1206905
:107D8000002802D02F46002511E000270FE0002236
:107D90008021204601F064FE002815D1002F15D067
:107DA0002168387888627F1C708A401E7082708AD1
:107DB000019B002806980090E9D10022402120462E
:107DC00001F04EFE002808D00320BDE72888216876
:107DD000C005C00D8862AD1CE6E7202060670299EF
:107DE00000200874B0E70220AEE77047014902485E
:107DF000C160FDE70400FA0500ED00E070B586B053
:107E000014216846FDF7D3F90F480124818B00291E
:107E100000D18483808B012805D0022801D100F095
:107E2000EDFB06B070BD0122084E95022946304692
:107E3000FEF7A9FD00210291039100950194694686
:107E40003046FEF7DFFCECE7D400002000040050D1
:107E500010B505242407002204212046FEF793FDD7
:107E6000002208212046FEF78EFD0A2002F00FF9BD
:107E7000012204212046FEF786FD0A2002F007F9C0
:107E8000002204212046FEF77EFD10BD10B505241A
:107E90002407002204212046FEF775FD0122082157
:107EA0002046FEF770FD0A2002F0F1F801220421BD
:107EB0002046FEF768FD0A2002F0E9F800220421BE
:107EC0002046FEF760FD10BDF8B5002405260746E4
:107ED00025463607002204213046FEF754FD0A20CD
:107EE00002F0D5F8012204213046FEF74CFD600671
:107EF000040E08213046FEF741FD002801D0641C25
:107F0000E4B2052002F0C3F86D1CEDB2082DE1D3F8
:107F1000002F03D0FFF79CFF2046F8BDFFF7B6FF08
:107F2000FAE770B5052605463607002204213046DB
:107F3000FEF729FD0024E80901D0012200E000221B
:107F400008213046FEF71FFD6806050E0A2002F0E4
:107F50009EF8012204213046FEF715FD0A2002F0AA
:107F600096F8002204213046FEF70DFD0A2002F0AB
:107F70008EF8641CE4B2082CDDD370BD10B5052466
:107F80002407012208212046FEF7FDFC01220421DE
:107F90002046FEF7F8FC002208212046FEF7F3FCFD
:107FA0000A2002F074F8002204212046FEF7EBFCC0
:107FB00010BD10B505242407002204212046FEF739
:107FC000E2FC002208212046FEF7DDFC0A2002F038
:107FD0005EF8012204212046FEF7D5FC012208218B
:107FE0002046FEF7D0FC0A2002F051F810BD70B513
:107FF00005252D070024012208212846FEF7C3FC91
:10800000062002F044F8012204212846FEF7BBFCBA
:10801000062002F03CF807E0641CE4B2FA2C03D915
:10802000FFF7C7FF012070BD08212846FEF7A6FC18
:108030000028F1D1002204212846FEF7A4FC0020EC
:1080400070BD0000F8B501F0D3FA01F00DFB564801
:108050000068C069554E564F800700D5FE60FDF799
:108060008DFE5449544D898F544C002929D05449D0
:108070000A7801218902002A05D0012A0ED0022A9D
:1080800010D0032A1DD1A08B01282DD0022818D191
:10809000454808213C38FFF78DFC12E0FF22F532FD
:1080A0009042F0D2A08B01281CD0022804D008E016
:1080B0002846FEF768FC04E03B4808213C38FFF7FF
:1080C00066FC0121C9023C48FEF758FC0025002847
:1080D0002CD03C480560FDF739FF2070A0790028BE
:1080E00004D007E00022E3E70122E1E70120A071CC
:1080F00001F014FD2078632806D9002208212E48BB
:10810000FEF741FC012205E0012208212A48FEF782
:108110003AFC002201210520C9030007FEF733FCC9
:10812000244C4034A08C012803D01CE0A57100220F
:10813000EBE725486946088072B680212348FDF7A1
:1081400049FD002804D0022269462048FDF7E6FDDB
:1081500062B61FA001F07EFDA58402F0DBFD642065
:1081600001F08EFFFE60608C012808D11148658403
:10817000058002F0CFFD642001F082FFFE60208CBC
:10818000012806D1258402F0C5FD642001F078FFA6
:10819000FE600848124A0188914202D1C088002836
:1081A00000D1FE60F8BD0000901500200400FA0523
:1081B00000ED00E0480D002000040050D400002035
:1081C000710000200C010020AAAA0000384A000813
:1081D000BDF8C8EBC9FDBCB6C4A3CABD0D0A0000FA
:1081E000AA55000010B53721202000F070F80321B7
:1081F000212000F06CF84021222000F068F80821CE
:10820000232000F064F8AA21302000F060F80A482A
:1082100001210187322000F05AF80121332000F0BB
:1082200056F85F21202000F052F8044800F008F8CA
:108230000A2001F02CFF10BD480D00200300002093
:1082400010B501460F2000F021F8002800D00120D1
:1082500010BD10B50446FFF791FE3220FFF761FE16
:10826000FFF7C5FEE0B2FFF75CFEFFF7C0FEFFF7C9
:1082700085FE3320FFF755FEFFF7B9FE0020FFF71C
:1082800023FE0446FFF795FE204610BD10B50C46B0
:10829000FFF7DFFF2070012010BD70B50D460446CA
:1082A000FFF76CFE3220FFF73CFEFFF7A0FEE0B2C6
:1082B000FFF737FEFFF79BFE2846FFF732FEFFF77A
:1082C00096FEFFF776FE0A2001F0E1FE70BD10B5C4
:1082D000FFF7E3FF012010BD10B50248FEF738FCA0
:1082E00010BD0000CC140020FEB50446002572B677
:1082F0000068394A831804D13849CD6803218904BC
:108300000D4081680191C168009141698669002B27
:1083100008D132484038836AC7043B438362836A8A
:10832000BB4383620846304348D02B482368C3428E
:1083300005D12A48C368032292049343C3600029ED
:1083400017D02068026901231A4302612068416145
:10835000FEF720FB0746FEF71DFB2168C01B0968DE
:10836000090703D47D21C9008842F4D92168082077
:108370004860002E17D02068016901221143016175
:1083800020688661FEF706FB7D270646FF00FEF7A4
:1083900001FB2168801B0968C90601D4B842F6D9DF
:1083A0002168102048600C482168C14206D10B4862
:1083B000C1680322920491432943C1602068016986
:1083C0004908490001612168019888602168009886
:1083D000C86062B6FEBD00000084FFBF40100240CE
:1083E0001CB5002116480091144A01910260C16336
:1083F0001205426081600722826301220261024607
:10840000C16020321170FF235170C2334362816218
:10841000117301638161042241634261C161FDF70F
:10842000AFFE084800908013019069460448FDF7AC
:1084300057FE00210248FDF7FDFD1CBD0024014050
:10844000701400200200000408B50848016B0122E6
:1084500011430163006B01211040009000220A20AB
:10846000FEF7A2FC0A20FEF795FC08BD00100240B2
:10847000F0B587B014216846FCF799FE4748C26AF8
:1084800004210A43C262C26A0A400592C16A802678
:108490003143C162C16A31400591C16A012421435F
:1084A000C162C16A21400591C16A02252943C162A6
:1084B000C06A22462840059005201C210007FEF7CF
:1084C00062FA012236493748FEF75DFA0022364942
:1084D0003448FEF758FA91210520002209020007CE
:1084E000FEF751FA314801900027052069460297AE
:1084F00000940007FEF786F90C20009011200190EF
:10850000032003900520029769460007FEF77AF9D9
:1085100010206A46039591C2052069460007FEF7C0
:1085200071F91120019002976946039700941D4844
:10853000FEF768F91E4801906946009502941948B3
:10854000FEF760F9E0020090694601970295154830
:10855000FEF758F91748694691C1694611480397D3
:10856000FEF750F991200002694691C10520694645
:1085700000070397FEF746F969460A4801970096F7
:108580000294FEF73FF9002201210520FEF70CFCC2
:108590000520FEF7FFFB07B0F0BD00000010024011
:1085A000010200000004005008300000000011101B
:1085B000000021100832000010B50F4C0D4820605B
:1085C000FF20053060600020A060E06020616061F5
:1085D000E0610121206249026062A161A06207207E
:1085E000E0622046FEF7F8FF206801684022114350
:1085F000016010BD00300140FC14002010B58AB0AD
:1086000000240494059406940794089401211848C2
:10861000099400940194029489070394016009214C
:1086200084604160046113494461C160FFF776F8DA
:1086300001200003049004A90D48FFF797F80C48A7
:10864000FFF78AF9089408A909480994FFF748F840
:108650006020009008480190029408226946039423
:108660000348FFF711F90248FFF7E8F80AB010BD18
:1086700054150020930400005702000000B585B097
:1086800014216846FCF793FD164815490160E12165
:108690004902416000218160C160016181610C2259
:1086A000C16142610162302141620121090381639C
:1086B0004900C163FFF734FA0120800200900220D4
:1086C00001900120029003200390042004900520D3
:1086D00069460007FEF796F801F01AFA05B000BDEA
:1086E0000038014090150020704700008307FF22EA
:1086F000DB0E9A408907090E994000280BDA000723
:10870000000F0838830808489B001818C369934372
:108710000B43C3617047830804489B001B1818680B
:10872000904308431860704700ED00E000E400E06B
:10873000BFF34F8F04490348C860BFF34F8F00BF9A
:10874000FDE700000400FA0500ED00E0F0B58DB093
:10875000962001F07FFF4B20C00001F095FFFF4FF6
:1087600000247C70B87B0C2801D30B20B873012245
:10877000052051020007FEF706F9B87B787378717F
:10878000F748BC70F74D00782870F7480221007850
:108790002871F648FEF7F2F8002865D00020B97974
:1087A000F04D49000843E871B86AE870401CB862AF
:1087B00078792946A8724200CE310846C338FCF7C2
:1087C000DDFC062068727879E94A80004119137847
:1087D000CB7252780A7329461339E04A0391937F8A
:1087E0000B75D27F4A75002213310F3002F01CF84E
:1087F0007879002180000F3002F028F8022001F083
:1088000079FFEC713C74BC7201203873FC72D9485A
:10881000FEF77EFA78840546BC707879FCF72EFF67
:10882000D54AD64BFCF724FE01F0C6FB0022D44B00
:10883000FCF76CFDFCF768FF0006C10C481980B21C
:108840000121C903B884884201D3401AB884CD48B5
:108850007863F878401CF870C648FEF759FA3884F7
:10886000C0484E300A9024E2012098E7C148FEF744
:108870004FFA3884C44DC54E21E0B87A002813D091
:1088800001F0A9FE059988420ED9049988420BD2BD
:1088900001F078FD3C73099801F0D5FE012001F04C
:1088A00029FF3872BC7211E0B248FEF731FA81B28A
:1088B0003984B88C814202D38019814206D30021C9
:1088C0000F2001F041FE2842F862D6D0F86A411C20
:1088D0007ED040047DD58122D20100210F2001F0FD
:1088E00078FF0021102001F02FFE41069D48490E1F
:1088F0000022503001F05EFE002001F0C5FE002095
:1089000001F077FE97485030417A0729ABD1022217
:108910009F49401DFCF756FC0028A4D190480078E0
:10892000FF2804D08F495031097881429BD100261D
:10893000354607A801F055FE042007AA310E2D0286
:108940000D433102165C0E43401EF7D5BE64FD6434
:1089500000263546104601F036FE042007A9320EE7
:108960002D02154332020E5C1643401EF7D53E65BC
:108970007D65B9786A46491CB9707A494D310D79DF
:1089800015724A7969464A720192787B00280AD1A9
:10899000012038710A897349CE310A8078710398B1
:1089A0000575019941756F486946CE30008809897F
:1089B000069188427ED10A987649008A08806948E3
:1089C00066494C30808A48836A48FEF7A1F901E085
:1089D0001DE163E13884788B6F49FF30C33080B28A
:1089E0003A46788388420CD94942401850836948F6
:1089F000694B01880B33491C89B20180994200D32D
:108A000004806649032008700A98544B81891986AE
:108A1000C0895886614B3A6B903B1A601A46B03A4F
:108A2000D37C1D072D0F032D00D07D741A09BA7455
:108A3000FC700125494ABD729186D0867879FF2164
:108A40009131484354493A6D593940180104C817C7
:108A50007B6D891858410206080A10435049099055
:108A60004018059019210998890240180490099826
:108A70003E46A843010E0002F165B0653948F36C2B
:108A80000A30B26C01F008FF3648736D1630326D53
:108A900001F002FF3348F36D1230B26D01F0FCFEBD
:108AA0003048082141722E490978017070798000A0
:108AB000002200E0ADE02B491C3001F0B5FE7079DA
:108AC000002180001C3001F0C1FE26492348F572C8
:108AD000042251314030FCF751FB2E48718B058840
:108AE0007D20C00068434018B0630B902D4801788A
:108AF000F1732D480E46C088FCF7A5FD029028466C
:108B0000FCF7A1FD0299FCF7C3FB7F21C905FCF727
:108B100066FBFCF7C1FD234980B20880711E8842C4
:108B200001D10120F872FD8414203E46385EFCF726
:108B300091FD00910890308CFCF7A0FD1B4A1C4B66
:108B4000FCF796FC054607910B98FCF783FD2A4637
:108B5000079BFCF77FFC009B089A2BE0600000203D
:108B6000D6000020BC110020D400002000040050DA
:108B7000F6000020CC140020666666666666E63F56
:108B800000000840A086010000D02724983A000089
:108B9000FC00002008010020E70300004C13002027
:108BA00000AEFCFFF4000020480D0020F853E3A5C0
:108BB0009B843E40FCF7AAFBFCF782FDF063BE48B5
:108BC000008800F0CBFAB07C012872D11222BB4998
:108BD000BB48FCF7D3FABB4C0822B949A01DFCF7EF
:108BE000CDFAB74920460A2208313630FCF7C6FADA
:108BF000E088B549401E884209D2E08E432806D25B
:108C0000002804D002F086F8642001F039FAFFF75A
:108C10008FFD0846FDF79EF8797B3E4688420DD3CE
:108C2000012131717179A54A491C717143006A3281
:108C30000699D15203990D75019A4A75A04A0321EC
:108C40000C3A11540A99A14A8B891386C989518615
:108C500082009A48316B9C308150B038C17C737C63
:108C60000807000F984202D9032800D07174934876
:108C7000736D643810181630326D01F00DFE707986
:108C80008E498000002264391C3001F0CDFD7079DE
:108C9000002180001C3001F0D9FD0AE02A460021A5
:108CA0000F2001F096FD387B002802D0002001F053
:108CB000A0FC398CBA8C914200D2D7E584481018B8
:108CC0008142FAD88348008881004018F9788842A8
:108CD00000D27C74804A00210F2001F07AFDB87820
:108CE0007871774800250C380078002812D1386C4C
:108CF000FDF7F4F80646794801883046FCF7F8F9A4
:108D00007748761E0088414388B26B490880BE834D
:108D100000F024FA0020B873797B3A798A1822E0AF
:108D2000674B0C3B195C00291BD0BC7BAB00641C5F
:108D3000BC73634C9C463C3CE150604B44006A333E
:108D40006E001C5B18339C5384001A335C4E1C5914
:108D500063466C3EF4506D1C33466033491EEDB2E1
:108D60001954401CC0B28242DAD8B878032801D224
:108D7000B87BB87355490022887B48730490401E25
:108D800034E000212EE04E4D8B006C3D5E19B44660
:108D9000EC587668B44223DD484F4D0082377F5B44
:108DA0000997474FA64694003C3F3F590597444FCB
:108DB0006C3F3C46FE504A3C2C190B9466884A3F57
:108DC0007E533C467A341E193D467A357468EC5021
:108DD000744663465C600B9C099F6780059F7760C3
:108DE000491CC9B28142CEDB521CD2B28242C8DBDE
:108DF0000020364C314D60729C35049A28E02F4992
:108E00002E4E43008231C95A6A36F15281006236D1
:108E10007658344F6E50BE4218D0294E3C3E76589C
:108E2000032E13D1677A0626BC467743234E491991
:108E30005036BE19214F6A37DB191B88B3800B8867
:108E4000F3804988674631817F1C6772401CC0B23D
:108E50009042D4D3194E552050363070AA207070ED
:108E60000420B070617A06204143881CF070B01C69
:108E7000891CFCF7FDFD2083617A062251438A1983
:108E800090803046891D00F037FE164A0020810090
:108E9000401CC0B26A500C28F9D30F4A002180321E
:108EA0000F2001F096FC0121052000224902000755
:108EB000FDF769FD0DB0F0BDDE000020201200209E
:108EC00058130020480D0020E70300006000002038
:108ED000983A0000E600002000D02724E20000209D
:108EE000E0000020FFFF010070470000F0B54A4994
:108EF00085B04848086001F0ABFE484800F0EEF845
:108F0000474C20834548801C00F0E8F860834348C4
:108F1000001D00F0E3F8434DA083FF2023302F46CF
:108F2000688040373979E1710491E88E3E49C0B2DA
:108F300008700390E88F2071A88F6071A87AA070E4
:108F4000A8880290A0622889FCF798FB374A384B22
:108F5000FCF78EFA01F030F80022364BFCF7D6F918
:108F6000FCF7D2FB86B2A681E888019031460090DA
:108F7000FCF7BEF8E08101460298FCF7B9F87143AE
:108F80008EB27D20C00066817043FCF777FB2A4AD1
:108F90002A4BFCF7D5FAFCF7B7FB2082A6827D208E
:108FA000C0000099FCF7A4F86082E083688F20720B
:108FB00004990120002902D120710A21217201990E
:108FC000002901D16421E980039A1749432A01D974
:108FD00043220A70B98A1A4A914201D90021B98202
:108FE000A989494261842084FCF7C8FEE082228A74
:108FF00014491548FDF790FE14A0A16A00F02AFE5E
:10900000E98816A000F026FE298919A000F022FEAA
:1090100005B0F0BD499B00085C000020004F00082F
:10902000D4000020480D0020160000206666666609
:109030006666E63F00000840F853E3A59B843E4087
:1090400010270000FF7F0000CC140020B1EAC7A960
:1090500049443A202564202E0D0A0000CDA8D1B63F
:10906000BCE4B8F43A202564206D732E0D0A00008C
:10907000B5A5B4CECDA8D1B6BBF9D5BECAFDC1BF8A
:109080003A202564B8F62E0D0A00000070B586B0AF
:1090900014216846FCF78BF801250F4EED030022E2
:1090A00029463046FDF76FFC012000240190029410
:1090B0006946009503943046FDF7A4FB0320019018
:1090C00002946946009503943046FDF79BFB02200D
:1090D00000F0D6FF06B070BD000400500088704755
:1090E00070470000F8B5044600206A461080194D0C
:1090F00055222A70AA226A700322AA70661DEE7099
:109100002A716971144A49008918AC712246E81D18
:10911000FCF734F8002007E029186A46897812889D
:1091200089186A461180401CB042F5DB611DA81CFD
:10913000FCF79EFC01466846018029190078C87139
:1091400068464078087221460931024800F042FB27
:10915000F8BD00000C140020480D002010B5134984
:109160000A8CCB8B9A4201D3D21A0A84104A098CFA
:10917000D2884A437D211018C90048430D49096827
:10918000401AFCF767FA0C4A0C4BFCF7D9F9FCF7CC
:1091900097FA0B49884201DD4A428018002800DA1C
:1091A000401808490968486110BD0000D40000203B
:1091B000480D00209C000020F853E3A59B843E400E
:1091C000FF7F0000CC140020034A1168382389B2C5
:1091D00099430143116070470030014010B5FDF71D
:1091E000DFFB10BD10B59AB034216846FBF7DFFFF6
:1091F00014210DA8FBF7DBFF1C2112A8FBF7D7FFFA
:109200001B4801680324E402A143C21489180160C9
:10921000FDF7D6FD17480169A143016106200090C2
:10922000FF200130029001200390102004900220C2
:10923000099040040B90000100240C900A946846A9
:10924000FDF7BCFF0F200D9003200E900F9410949B
:10925000012111940DA8FDF79FFE8120129003209B
:1092600080041890149412A8FDF7E4FD1AB010BD04
:109270000070004040100240104801688215114300
:109280000160C1680E4A1140C16001680D4A114079
:1092900001608168490849008160016801229204E7
:1092A00091430160C168FD2212049143C160002115
:1092B00001610649044888607047000000100240C0
:1092C0000C40FF88F6FFF6FE0050000800ED00E0BD
:1092D00070B5026801239B07114C124D984203D0D0
:1092E000A04201D0A84203D17026B2434E68324357
:1092F000984203D0A04201D0A84204D103231B020C
:109300009A43CB681A4380239A430B691A4302603D
:109310008A68C262096881620121416170BD0000F2
:10932000000801400014014010B5CB06DB0E0121FE
:10933000046A99408C430462016A9A4011430162B5
:1093400010BD30B58468FF252D021B021343AC43CA
:109350000B432343836030BD826870239A430A43E2
:1093600007210A438260704730B5026A52085200F2
:109370000262026A456883697024A3439C080B68F3
:10938000A40023430224A2438C68456014438361F4
:1093900049684163046230BD30B5026A10239A43C4
:1093A0000262036A4568826973242402A2430C683E
:1093B00024021443202293438A68456012011A4311
:1093C000846149688163026230BD30B5026AFF235F
:1093D00001339A430262026A4568C3697024A34359
:1093E0009C080B68A400234301246402A2438C68F8
:1093F000456024021443C3614968C163046230BDFF
:1094000030B5026A01231B039A430262036A45686E
:10941000C26973242402A2430C682402144301226B
:10942000520393438A68456012031A43C461496832
:109430000164026230BD30B5036A046A64086400E6
:1094400004628469F025AC43120122430A24A34339
:109450000B438261036230BD30B5036A1024A3431D
:1094600003628469036A0F252D031203AC43224370
:10947000A024A343090119438261016230BD0000A9
:1094800070B501F075F80D4C0D4D606402E001F00F
:109490006FF86064A842FAD10020E08220780028AA
:1094A00009D0012802D0022805D102E0FCF782FC95
:1094B00001E0FFF74BF900F04DFF70BD60000020A8
:1094C0003001CADE10B5818CC90707D001684A682F
:1094D00001235B049A43836A1A434A60818C89079B
:1094E00007D501684A6801231B049A43C36A1A43DB
:1094F0004A60818C490707D501684A6801239B04AB
:109500009A43036B1A434A60818C090707D50168A7
:109510004A680123DB039A43436B1A434A60818CF8
:10952000C90607D50268916801231B039943836B21
:1095300019439160818C890607D501688A680123E7
:109540005B039A43C36B1A438A60818C490612D528
:1095500003685A6801210905046C8A4322435A6052
:10956000026C8A4207D10268516803235B05994364
:10957000436C19435160818C090607D501684A681C
:109580000123DB04806C9A4302434A6010BD000053
:10959000F8B500260446C667FDF7FCF905462068C5
:1095A0000068124F000709D501212B46002249050A
:1095B0002046009700F054FA00280DD1206800687A
:1095C00040070BD501212B46002289052046009734
:1095D00000F046FA002801D00320F8BD2020606783
:1095E000A067603426740020F8BD0000FFFFFF0173
:1095F000F8B5184CC826E078002829D160790028F1
:1096000026D101206071144D686B002700281ED000
:10961000686BC821081A15E01048E168405C616970
:1096200088470F480A21008848430E490880E068AF
:10963000401CE060E068C82800DBE760696BC82078
:10964000401A761EE168814201D0002EE4DC677189
:10965000F8BD00004800002000000240800C0020FF
:10966000E6000020F800002070B5224CE0780028C9
:109670003FD1207900283CD1012020711E4EF16994
:1096800000250906002933DA2156625791420AD192
:10969000F06940062CD5A079002829D0A571208931
:1096A000401C208124E0A179002903D1A0710A2067
:1096B00000F0EDFC00202056CC2148430F49421811
:1096C000206912181279B262401C00222061A25651
:1096D000CC235A43895881420ADC25612078401CFA
:1096E000207020780E2800D12570A078401CA07032
:1096F000257170BD4800002000380140580100204D
:1097000010B5806A0022014640314A834A82FEF742
:1097100068F910BD70B5846A606FA56F21688968AB
:1097200000260906002906DA212804D15220065312
:10973000204600F047F820688068400606D5222DB4
:1097400004D15A200653204600F02CF8E06F102177
:109750000843E0672046FEF744F970BD10B50146A6
:109760000968806A0968890614D400225A210A52BD
:1097700001680A68FF2301339A430A6001688A6816
:10978000520852008A6001688A6840239A438A60BE
:1097900020218167FEF7C0FA10BD10B5806AFEF780
:1097A000BCFA10BD01680A68FF2321339A430A609E
:1097B00001688A68520852008A602021816700216E
:1097C0000166704701680A68C0239A430A60202135
:1097D0004167704770B5164CE278002A0CD12279A7
:1097E000002A09D10122E2700025C82903DC0222E7
:1097F000A256002A01DCE57070BD0123E356CC229D
:1098000053430C4AD1500123E356CC2673439B1893
:109810000A460146181DFBF7B1FC6078401C6070D9
:1098200060780E2800D16570A078401EA070E2E735
:109830004800002058010020F8B504462669A268B7
:10984000E76932436669102000253E4323683243AE
:1098500078491E68784F3E4016431E6023685A6858
:1098600003263603B243E66832435A602368A2698E
:109870008B4201D0266A32439E680B273F02BE43CB
:1098800016439E606D4E23686D4AB3420CD1D26878
:109890009207920F06D0012A38D0022A34D0032A28
:1098A00020D11EE001201DE0664EB3420AD1D268ED
:1098B0000C26324026D0042A28D0082A24D00C2A8C
:1098C00010D10EE08B420DD1D668032292021640D1
:1098D00018D001229202B61A18D0B61A14D09642A5
:1098E00000D10820564A0126403A574FF6038B42D2
:1098F00036D100280CD002280DD0042812D0082818
:109900001FD11CE00020EDE70220EBE70420E9E78F
:10991000FDF7F8FB08E01068C00601D5384605E001
:109920004A4803E0FDF70EFC002873D0626851003E
:109930005118814205D81103814202D303E0304619
:10994000F4E7012566E0010E0602500800233018F6
:109950005941FBF7E3FB03210902411A3C4A55E058
:10996000E169B14232D1030000F09BF909070A0D09
:1099700006250606062B0600E3E7FDF7C3FB1CE001
:10998000FDF7D0FB19E010686168C00602D54808F1
:10999000304A01E0304A48088018FBF7A9FB80B242
:1099A00001462E4A10399142CBD8511C0140000784
:1099B000400F08432CE0FDF7C5FB616840004A08F2
:1099C000EAE76168012248081204E5E7030000F0B5
:1099D00068F909070A0D06260606062C0600B0E7F8
:1099E000FDF790FB1DE0FDF79DFB1AE01068616834
:1099F000C00602D54808C01902E014484A081018E9
:109A0000FBF776FB80B20146144A1039914298D890
:109A10002168C8600020206660662846F8BDFDF712
:109A200091FB61684A088018EAE761684808801974
:109A3000E6E7000000480040F369FFEF003801400E
:109A4000401002400044004000093D000024F400A2
:109A5000FFFC0F0000127A000048E801EFFF000051
:109A6000FFB581B017460E4604460A9D09E0681C02
:109A700007D0FCF78FFF0499401AA8420CD8002D9C
:109A80000AD02068C1693046884318D00020B84207
:109A9000EDD0002005B0F0BD20680168FF22A132A2
:109AA0009143016020688168490849008160202055
:109AB0006067A0670020603420740320EAE701207B
:109AC000E5E7000010B50449102009680862024863
:109AD000FDF788FF10BD00009015002001B501239F
:109AE0001A4669460248FEF719F90248C06908BDDE
:109AF000901500200038014070B50D460646002440
:109B000003E0305DFFF7EAFF641CAC42F9DB70BD97
:109B100001490D20887070474800002010B50748A3
:109B20000A22418A51438184FEF78EFCFEF7A6FD8E
:109B3000C82203490348FEF793F810BDD400002063
:109B4000800C002090150020F8B53D4C00232178B2
:109B50003C4A1D46082910D0072945D006294ED079
:109B6000052950D0042951D0032952D0002954D0BE
:109B7000012956D0022958D059E0A17800264A1F61
:109B800004E0304FBF5DFB189BB2761C9642F8DBB9
:109B9000667927799A195118E3786278C918891873
:109BA000C9194018C0071AD0012E14D0022E16D1A0
:109BB00025482449C018FBF7E1FA01F0ABF864200E
:109BC00000F05EFABFF34F8F21492048C860BFF311
:109BD0004F8F00BFFDE759081046FFF783FA257045
:109BE000E570A570A571F8BDA1795054491CC8B2A3
:109BF000A071A178491F8842F5D1082001E060706A
:109C000007202070F8BDE0700620FAE7607105209B
:109C1000F7E7A070E5700420F3E7552807D101208D
:109C2000EFE7AA2803D10220EBE7032803D0257031
:109C3000E570A570F8BD032020702071F8BD00000C
:109C4000CB000020A8130020480D00200400FA05D6
:109C500000ED00E00FB410B503A9044B044A0298CC
:109C600000F002F910BC08BC04B01847B1A8000805
:109C7000180100202021020C01D010211046020AF8
:109C800001D010460839020901D01046091F820888
:109C900001D01046891E420801D0881E7047081A5C
:109CA000704730B47446641E2578641CAB4200D201
:109CB0001D46635D5B00E31830BC184702E008C82E
:109CC000121F08C1002AFAD170477047002001E036
:109CD00001C1121F002AFBD1704708B50021684658
:109CE00001706B46012202212C2000F081FD02212F
:109CF000684601706B4601222C2000F079FD08BDFA
:109D000038B504466D20694608706B460122074944
:109D10002E2000F06DFD0649002C01D0054A00E020
:109D2000054A2E2000F04AFD38BD0000060800005C
:109D300006180000070600000716000038B50446A4
:109D40006B4602220021362000F018FCB3212300CC
:109D5000FFF7A7FF0E0F08153A3A3A3A1C273A3A8E
:109D60002F34483A00216846017040784108490084
:109D700014E06946087880088000401C04E06946C9
:109D8000087880088000801C08701DE06846027812
:109D90000A40483202704178802001436846417091
:109DA00012E0684602780A40027040784106490E87
:109DB000F4E7694648780221084303E06946487899
:109DC000FD210840694648706B460122002136207B
:109DD00000F00EFD012200AB11463620013300F0E9
:109DE00007FD38BD69460878CF2108406946203014
:109DF000CAE708B5032168464170012101706B462E
:109E000002220021362000F0F3FC0122D2030621B9
:109E10002D2000F0D3FC012000F032F90120FFF7E3
:109E20008DFF08BD08B5020A69464A7008706B4686
:109E3000022204212D2000F0DBFC0320694608707B
:109E40006B46012206212D2000F0D2FC002069463D
:109E500008706B46012206212D2000F0C9FC0A2162
:109E60002D2000F071FB08BDFFB58DB00446002524
:109E700006E025280AD0109A0F999047641C6D1CA3
:109E800020780028F5D1284611B0F0BD0027012127
:109E9000484A009700E00743641C23780846203BAB
:109EA00098401042F7D120782E2817D1042007437C
:109EB0006078641C2A280CD10E98641C02C800919A
:109EC0000E900BE000990A22514330394018641C6F
:109ED00000902078014630390929F3D920780028EC
:109EE000D1D0642808D0692806D075281ED0109AD1
:109EF0000F9990476D1C5BE00A200E99019001C9F3
:109F00000E91002802DA40422D2102E0390504D5E5
:109F10002B216A461172012103E0F90704D02021A8
:109F2000F7E70BAE0B910DE00021FAE70A200E993E
:109F3000019001C90E91F7E70199FBF7D9F830318B
:109F4000761E31700028F7D103A8801B20300190C5
:109F5000780701D5009801E001200090019988421E
:109F600001DD401A00E000200027009006E002A872
:109F7000109AC05D0F9990476D1C7F1C0B9887420B
:109F8000F5DB04E0109A30200F9990476D1C009982
:109F9000481E00900029F5DC05E03078109A761C08
:109FA0000F9990476D1C0199481E01900029F4DC1F
:109FB000641C65E709280100F8B54A002B4B520DD7
:109FC000D6182B4A0C460546142E2BDA002E12DA30
:109FD000284BFBF79BF900221346FBF7C1FC40D24C
:109FE000002C03DA0124E40700253AE02046284348
:109FF00037D0214C14E0214F0B46F7403B402B4318
:10A0000031D01C4BFBF782F900221346FBF7A8FC6A
:10A0100027D2002C03DD01200005F0400419BC43C9
:10A0200000251EE0332E1EDC33460027143BFF4381
:10A03000DF40384217D00F4BFBF712FA00221346CD
:10A04000FBF78EFC0DD2002C0ADD142E0CD0342030
:10A05000811B012088404019A84200D2641C05469B
:10A06000BD4321462846F8BD641CF9E701FCFFFF0B
:10A070009C7500883CE4377E0000F03FFFFF0F0036
:10A080007D2110B5C900484300F001F810BD002142
:10A0900040E000BF00BF00BF00BF00BF00BF00BF67
:10A0A00000BF00BF00BF00BF00BF00BF00BF00BFB8
:10A0B00000BF00BF00BF00BF00BF00BF00BF00BFA8
:10A0C00000BF00BF00BF00BF00BF00BF00BF00BF98
:10A0D00000BF00BF00BF00BF00BF00BF00BF00BF88
:10A0E00000BF00BF00BF00BF00BF00BF00BF00BF78
:10A0F00000BF00BF00BF00BF00BF00BF00BF00BF68
:10A1000000BF00BF00BF00BF00BF00BF00BF00BF57
:10A1100000BF491C8142BCD370470000FEB5044615
:10A120000020019000906079734940000E5A6178D8
:10A130002578491E7148CFB20163042D77D0072DD1
:10A1400075D000210291217801736C49E3790122D5
:10A1500092058969002B6CD0914381616748217A0F
:10A160004173217A82698907890B0A438261002140
:10A17000042000F02EFB324661492E2000F01EFB29
:10A180003846FFF7BDFD5F4E0522705D8100401827
:10A190005D49431807212B2000F02AFB5B490298F8
:10A1A00001220B180B21282000F022FB705D58497A
:10A1B00080000A580C21282000F00BFBE07955495B
:10A1C00080004018A1794900425A0221272000F05E
:10A1D000F5FA51487E00825B0421272000F0EEFA58
:10A1E000E079002829D0A07804282CD028206946BE
:10A1F000087220220621272000F0E0FA02AB01229B
:10A200002621272000F0F4FA444938014018E1786B
:10A21000890042580821272000F0DBFAA17A601C4F
:10A22000627A0902114313D016E000E001E0012137
:10A2300088E71143F608816190E764220621272010
:10A2400000F0BCFAE0E71020694608720246D1E748
:10A2500033490172090A4172417A007A0A020243C3
:10A260002021272000F0AAFA2E4F0C2123203A6843
:10A2700000F0AFFAF01982880421232000F09EFA42
:10A28000A07900280BD0E07927490122431800214A
:10A29000212000F0ADFA03200190012000902A0750
:10A2A000120F10010243607800218007000B024367
:10A2B0000198000502430098400402432079C0063B
:10A2C000400902436079C00602431F2000F081FA72
:10A2D000A07861780123084302040848DB03026187
:10A2E000E179490319430A4302610021082000F083
:10A2F00070FA0020FEBD0000ECAD00081C0100203B
:10A300000428000094AD000817000020350000204C
:10A310009CAD0008BCAD0008C8AD0008CCAD00087D
:10A3200041100000B4AD00083700002038B50C46DD
:10A3300007498A8B002102432C2000F03FFA68462F
:10A3400004706B46012206212C2000F051FA38BD22
:10A350001C01002010B5FFF7C0FC10BD10B504466D
:10A360000421362000F0F0F80121C902002C01D0B0
:10A37000084300E0884302460421362000F029FA11
:10A3800010BD000038B540206946087000210E203D
:10A3900000F0DAF80446002211460E2000F019FA07
:10A3A0006B46012200210D2000F022FA074A00210D
:10A3B0000F2000F00EFA00F0E7F9224600210E20EF
:10A3C00000F007FA02480021017338BDF8FF272486
:10A3D0003C0100207CB505460420694608704B4CC2
:10A3E0000020607521462031206348710873A083E6
:10A3F0006063A06300F0BCF8454E206002E000F00E
:10A40000B7F82060B042FAD10020FFF797FC41482E
:10A410000078242801D9243806E00621FAF768FEDE
:10A420000622101A40010843020601040A430102F1
:10A430000A43024300211E2000F0CBF96B460122A3
:10A440000021242000F0D4F91E20FFF7EBFC86B297
:10A45000300AA0730420FFF7E5FC0006000E0DD0C3
:10A4600002206946087101AB012212212D2000F063
:10A47000BFF9A08B012109030843A08300F078F8FD
:10A4800020600620FFF7CEFC60600720FFF7CAFCC3
:10A49000A060F006C00E207501D110202075C0B25A
:10A4A00000F0E2F9E80707D0FFF7A3FCA08B012139
:10A4B000C9020843A0830AE00521362000F02EF8E7
:10A4C0001549084002460521362000F077F90120A1
:10A4D000FFF734FC0021042000F036F8A0610021D1
:10A4E000262000F031F81521890308430246002197
:10A4F000262000F06EF900222621362000F05EF9B9
:10A5000000F036F8206000207CBD00001C01002017
:10A510003001CADE16000020FFFD000038B5094CEE
:10A5200089B280B26B46022200F028F8002806D1DA
:10A5300068464078010268460078081884B22046D0
:10A5400038BD0000FFFF000038B50024E44389B2A5
:10A5500080B26B46042200F011F8002806D10321D6
:10A560006846435C2202D418491EFAD5204638BDFD
:10A5700010B500210846FFF7E7FF10BD38B50029E8
:10A5800009D0402420436C462070C8B27F2906D8E9
:10A59000607002200AE069460870012006E080240D
:10A5A00020436C466070C809A0700320694600F023
:10A5B0008BFB38BD10B5144603460A4621461120D0
:10A5C000FFF7DCFF10BD10B5034605220021152062
:10A5D000FFF7D4FF10BD10B501210620FFF7B4FF2F
:10A5E00010BD10B50346052200211720FFF7C6FF56
:10A5F00010BD38B5054600206946087000F0C4F863
:10A60000FF2401342246002D01D003221202002132
:10A610000D2000F0D3F8002D13D06B46012203214A
:10A620000F20FFF7ABFF68460078000709D5FFF75A
:10A63000A9FE224600210D2000F0C0F80020C043F2
:10A6400038BD002038BD10B5024601210A2000F0B7
:10A65000C0F810BD10B5044600211A20FFF774FFA2
:10A66000000D22030005120B024300211A2000F006
:10A67000B0F810BD10B5024602492E2000F09EF839
:10A6800010BD000004180000F8B505466B46012215
:10A6900003210420FFF772FF0126114C3607002D1D
:10A6A0000DD02A4600210C2000F088F86946087871
:10A6B0001021084369460870A069304307E06946E5
:10A6C0000878EF21084069460870A069B0430B463E
:10A6D000A06101220321042000F08AF8F8BD0000E7
:10A6E0001C01002010B502460021182000F066F879
:10A6F00010BD0000F8B50746002568460570B8078C
:10A70000204C2E4600280ADA8020694608706B46E5
:10A71000012200210D2000F06BF801202073F807C2
:10A720006946087821D006210843694608706B46BF
:10A73000012200210D2000F05BF803210F20FFF71C
:10A74000EDFE8121C900084219D0402069460870F9
:10A750006B46012200210D2000F04AF80020FFF78F
:10A76000FDFD00252673ED4309E0022108436946FB
:10A7700008706B46012200210D2000F039F82846B0
:10A78000F8BD00003C0100201CB56B4601220321EE
:10A790000F20FFF7F3FE684600784022C109104001
:10A7A000C9014000814208D0012069460871024673
:10A7B00001AB03210D2000F01BF81CBD08B56B4652
:10A7C0001A70120A5A7089B280B2022200F010F890
:10A7D00008BD38B500236C46E254120A5B1C042BFA
:10A7E000FADB89B280B22346042200F001F838BDBA
:10A7F00038B58024002909D0C02528436D4628702B
:10A80000C8B27F2907D86870022009E02043694652
:10A810000870012004E020436870C809A870032074
:10A82000694600F093FA38BD10B51446012312189A
:10A830009B029A4202D90020C04310BD0B46821EE3
:10A8400021460920FFF7D4FF002010BD10B5054AAE
:10A850008905126901430A4300210820FFF7B9FF67
:10A86000002010BD1C01002038B504466B460122B3
:10A870000E212B20FFF782FE68460078E106400992
:10A880004001C90E0143684601706B4601220E214A
:10A890002B20FFF7ADFF38BD10B5002142541C0638
:10A8A000120A22431B0A491C0429F7DB10BD0000D1
:10A8B00013B501231A4669460248FDF72FFA00989E
:10A8C0001CBD000090150020FCF772F8FEF78AFC12
:10A8D000FDF7CEFD41494248002522C00560856153
:10A8E000C56140490562C1600838FCF797F9FDF77A
:10A8F000ABFDFDF7C3FEFDF75FFEFDF771FD05261D
:10A9000001223607D1033046FCF73DF8FEF7EEFA98
:10A91000FBF790F8FBF702F9FBF7DAF8FDF76EFAB0
:10A920000721B015FFF702FDFFF714FD2E4C0A2199
:10A93000608A01224843A08411033046FCF723F8C3
:10A940002748C8222949C430FDF78AF9284F294EE3
:10A95000E07800283FD0E07900283CD0FEF742FCA8
:10A96000E570FBF7F3FA20700F280AD901221103D2
:10A970003046FCF708F8FEF783FD002201210903A9
:10A9800009E0012251033046FBF7FDFFFEF778FD99
:10A990000022012149033046FBF7F5FFFDF752FB8A
:10A9A000A08C002801D0401EA0841348A18C007800
:10A9B0000843CDD13878002801D00328C8D101211F
:10A9C000C9023046FBF7DAFF0028C1D10121084651
:10A9D000FCF716FABCE7FDF735FBB9E7007C004051
:10A9E000CC140020FFFF0000D4000020800C0020C9
:10A9F00071000020000400504E00002010B586B009
:10AA00001748FCF790F814216846FAF7D0FB154870
:10AA10000090032001900020029005206946000765
:10AA2000FBF7F0FE69461048FBF7ECFE69460F485D
:10AA3000FBF7E8FE01210846FCF7E2F9FF240134A8
:10AA40002046FCF7B5F90A4908680422104308605B
:10AA50002046FCF7BDF9FCF7C3F906B010BD0000B5
:10AA6000CC140020FFFF000000040050000800503C
:10AA70000070004010B50446FDF780FA4E20FDF747
:10AA800050FAFDF7B4FAE0B2FDF74BFAFDF7AFFA72
:10AA9000FDF774FA4F20FDF744FAFDF7A8FA0020FD
:10AAA000FDF712FA0446FDF784FA204610BD70B592
:10AAB0000D460446FDF762FA4E20FDF732FAFDF727
:10AAC00096FAE0B2FDF72DFAFDF791FA2846FDF768
:10AAD00028FAFDF78CFAFDF76CFA0A20FFF7D7FA8F
:10AAE00070BD000010B52421002000F04DF81B4877
:10AAF000FFF7CDFA00210F2000F046F805211020C5
:10AB000000F042F80421112000F03EF883217F205C
:10AB100000F03AF869217F2000F036F8BD217F204F
:10AB200000F032F80E480078262804D10022402197
:10AB30008C2000F019F8012000F02AF809481421AF
:10AB40000187282000F020F80A20FFF7A0FA012052
:10AB500000F036F8012000F043F810BD204E000050
:10AB600000000020480D0020F8B517460E460546A7
:10AB70000024FFF77FFF3946B44331402143284684
:10AB800000F002F80020F8BD10B5FFF790FF10BDEF
:10AB900010B500280AD000212720FFF7F5FF042177
:10ABA0001920FFF7F1FF8721162005E0002116206C
:10ABB000FFF7EAFF00211920FFF7E6FF10BD0000B4
:10ABC00010B5002801D0002200E080228021112051
:10ABD000FFF7CAFF0148FFF75AFA10BDA08601002F
:10ABE00010B5002811D001212F20FFF7CDFF6221E1
:10ABF0003020FFF7C9FF46213120FFF7C5FF322182
:10AC00000846FFF7C1FFA22100E022213320FFF711
:10AC1000BBFF10BD0C480D4A0188914210D1C1887C
:10AC200032290DD3C18E43290AD8818F012907D833
:10AC3000C08F012804D8044840308088012801D9F9
:10AC40000120704700207047480D0020AA550000E1
:10AC500010B50122920219491948FAF7D5FF174891
:10AC6000184902888A4227D0018004218180FF216F
:10AC7000F531C1800A21018100211E224181D24388
:10AC800082810122C2810184018241828182C1824A
:10AC9000018381834323C386022303877823438769
:10ACA0008287C2870246403291829180118451840A
:10ACB0009184C18300F02EF810BD0000480D0020E3
:10ACC00000FC0008AA550000F0B58C4600251026AF
:10ACD000052109078E620E4C08E067467F5DE7603C
:10ACE000A768FF07FCD0E7681F706D1C8542F4DB86
:10ACF0000020074606E0E760A568ED07FCD0E568A0
:10AD00001D54401C9042F6D38E610020F0BD00001F
:10AD10000030014070B5FFF77DFF002801D0012011
:10AD200070BD72B60124074DA40221462846FAF7E9
:10AD300051FF002804D0224603492846FAF7EEFFC7
:10AD400062B670BD00FC0008480D0020F0B500257B
:10AD5000102605279C463F070B46BE620C4C06E0BA
:10AD6000595DE160A168C907FCD0E1686D1C8542AE
:10AD7000F6DB002007E06146095CE160A168C907D5
:10AD8000FCD0E168401C9042F5D3BE610020F0BDCC
:10AD9000003001400000010203040005405C000097
:10ADA000A05C0400C06C0800805C0400E03F1E0052
:10ADB000E07D1E0007A9022570889B880A00160006
:10ADC000010006000100020087008D002D001A31ED
:10ADD00052001A339A001A351D011A376B003B31A5
:10ADE000BE003B335E013B3596023B37000099596C
:10ADF0009959EB518F421E45142E0080EB51F528D6
:10AE00003333E13A703DE13AC235852BC2353333F5
:10AE1000C235C235AE47E13A5138A330513800004F
:10AE200000000000000001020304060708090304F3
:10AE300006080C1018203000000000010203040076
:10AE400060AE0008000000201C010000BC9C00084F
:10AE50007CAF00081C0100209C190000CC9C00085D
:10AE600027000000000000000000000000000000BB
:10AE700000000000000000070400091E080540084B
:10AE800026091040085608054008261D040008BE83
:10AE90001D040008BED8BC401008000001000000DE
:10AEA0000000C84200000000000000000000000098
:10AEB0000000000000000000000000000000000092
:10AEC0000100000000000000000000000000000081
:10AED000000000008C0A00000000000000000000DC
:10AEE0000000000000000000000000000000000062
:10AEF0000000000000000000000000000000000052
:10AF00000000000000000000000000000000000041
:10AF10000000000000000000000000000000000031
:10AF20000502140009090102008100000000000070
:10AF30000100000000000000000000000000000010
:10AF40000000000000000000000000000000000001
:10AF500000000000000000000000000000000000F1
:10AF600000000000000000000000000000000000E1
:0CAF7000000000000000200000000000B5
:04000005080050C1DE
:00000001FF
